:1000000000308A0058280000831A0A28A500030E31
:10001000A6000F288312A500030EA600A6140A0846
:10002000AD008A018313A50E0408A7002008A800CC
:100030002108A9002208AA002308AB002408AC006C
:1000400083128C308400801E27288C1A3C282708B5
:1000500084002808A0002908A1002A08A2002B0873
:10006000A3002C08A4002D088A00260E830083120A
:10007000250EA618831609008C1E3C281A08AE000F
:100080002E0886008C128A1127283330840000083D
:10009000031957280630A100A001A00B4D28A10B81
:1000A0004C287B30A000A00B5328800B4A2800343A
:1000B00084011F308305813083169900A630980093
:1000C00090308312980083161F149F141F159F11E0
:1000D0008312AF01B001B101B201FF308316850078
:1000E000860183128601831607148714C030831299
:1000F0008B0483168C1683120508300203198D2891
:100100000508B000C030AF050508AF042F080C1E6D
:10011000872899000A30B3004520003007180130C5
:1001200031020319A428B1010718B10A310B9A282A
:100130002F179D28B10803192F132F080C1E9E2876
:1001400099000A30B3004520003087180130320290
:100150000319BB28B2018718B20A320BB128AF17B6
:10016000B428B2080319AF132F080C1EB528990044
:0A0170000A30B30045207C2863002C
:02400E007A3FF7
:00000001FF
